:020000021000EC
:10E0000058C000008FC000008DC000008BC0000011
:10E0100089C0000087C0000085C0000083C00000E8
:10E0200081C000007FC0000060C500007BC0000010
:10E0300079C0000077C0000075C0000073C0000008
:10E0400071C000006FC000006DC000006BC0000018
:10E050006AC0000067C0000065C0000063C0000027
:10E0600061C000005FC000005DC000005BC0000038
:10E0700059C0000057C0000055C0000053C0000048
:10E0800051C000004FC000004DC000004BC0000058
:10E0900049C0000047C0000018034400650061004B
:10E0A0006E002000430061006D0065007200610099
:10E0B000000011241FBECFEFD0E2DEBFCDBF04B6FB
:10E0C00003FE19C0809181019091820182549C4D80
:10E0D00091F484B7877F84BF88E10FB6F89480936A
:10E0E0006000109260000FBE1092820110928101B8
:10E0F000E0E0F0E0099511E0A0E0B1E0EEECFEEE2A
:10E1000001E00BBF02C007900D92A436B107D9F70A
:10E1100011E0A4E6B1E001C01D92A138B107E1F71A
:10E1200072D3D3C66DCF1F920F920FB60F921124E8
:10E130008F9380E489B98F910F900FBE0F901F903D
:10E140001895282F17C08091F2009091F300892B29
:10E1500071F48091E8008B7F8093E80003C08EB358
:10E16000882351F08091E80082FFF9CF02C08091AE
:10E17000F1002150222339F7089520917301309145
:10E18000720180917101909170018093650190936B
:10E190006601C901809367019093680108951F93F8
:10E1A000DF93CF9300D000D000D0CDB7DEB7809101
:10E1B0006B018823D9F080916E01843049F48091FD
:10E1C0006F01882339F4809170018F3F19F40EC0DC
:10E1D000853061F08AE08093000183E080936A01DA
:10E1E0008091EB0080628093EB00FDC080916E0116
:10E1F000843009F45EC0853030F4813059F08330CA
:10E2000009F0F1C022C0853009F4BAC0863009F0A7
:10E21000EAC0DDC010916F01123008F0E4C0ADDF3C
:10E22000112389F48091650190916601A0916901A3
:10E23000B0E023E0FC01A0935B0020935700E89539
:10E2400007B600FCFDCF85E008C080916F018823F0
:10E2500011F0823029F491DF89E080930001C3C07E
:10E26000813009F0C0C020E030E040E050E04BBF1A
:10E27000F90187918F3F81F0CA01AA27BB278093BC
:10E28000690130936601209365018AE08093000163
:10E2900085E080936A01A7C02F5F3F4F4F4F5F4FCC
:10E2A000203080EE380781E0480780E05807F9F613
:10E2B0009AC080916F01833081F581E08093640181
:10E2C0008091740190917501892B71F0809170019A
:10E2D000813009F088C08091730190917201909310
:10E2E0006D0180936C017FC080917001882391F44F
:10E2F00082E49CED90938201809381012CE088E17F
:10E3000090E00FB6F894A895809360000FBE20931C
:10E31000600069C01092010166C0882309F063C0E3
:10E32000809170018F3F09F05EC080E090E0A0E036
:10E33000B0E033E025E0FC01A0935B003093570090
:10E34000E89507B600FCFDCFFC01A0935B0020938D
:10E350005700E89507B600FCFDCF80509F4FAF4FA8
:10E36000BF4F803040EE940741E0A40740E0B4077F
:10E3700011F781E180935700E89510926B0133C04B
:10E38000DE011196E5E0F1E083E001900D9281500D
:10E39000E1F7DE011496E2E0F1E083E001900D92F6
:10E3A0008150E1F79091700180916F01882329F4E9
:10E3B000FE01E90FF11D818107C08130A1F4FE014A
:10E3C000BC97E90FF11D8081809376010CC080918C
:10E3D0006F01833041F480917001882321F4809192
:10E3E00071018093690126960FB6F894DEBF0FBEC7
:10E3F000CDBFCF91DF911F9108958F929F92AF92E1
:10E40000BF92CF92DF92EF92FF920F931F93CF9321
:10E41000DF93809179018F77813209F0E7C180E441
:10E4200089B9C0917F01D0918001D0937501C093CB
:10E43000740180917A01833009F4A2C1843030F4F0
:10E44000813071F0823009F0D1C106C1853009F404
:10E45000B5C1853008F4AAC1863009F0C7C1BDC175
:10E460008091E800877F8093E80080916401882391
:10E4700019F095DE10926401209729F42DC08EB317
:10E48000882309F4B3C18091E80082FFF8CF80911E
:10E49000F10080936E019E01215030403093750150
:10E4A00020937401EFE6F1E00CC08091F1008193BC
:10E4B0002150304081E0E437F80719F4318320839C
:10E4C0000AC08091F2009091F300892B71F730938C
:10E4D00075012093740163DE80910001853009F09D
:10E4E000B7C08091740190917501892B21F482E06D
:10E4F00080930001ADC08AE124DEC0916501D09116
:10E5000066019E012F71822F1CDEA0906701B090E2
:10E5100068010894A11CB11C85010C1B1D0B0894FB
:10E52000A108B10880916F01882309F08CC06801AF
:10E53000D694C794CE01A0916901B0E07C018D0111
:10E54000A8019701A0E08824839465E0962EB3E0AB
:10E5500047C08091F2009091F300892B71F4809173
:10E56000E8008B7F8093E80004C08EB3882309F411
:10E570003DC18091E80082FFF8CF0894C108D1081E
:10E580008091F100682F8091F100782F0B01F90143
:10E5900040935B0080925700E8951124AF5F2E5F97
:10E5A0003F4F4F4F5F4FA03819F0C114D104C1F451
:10E5B000F70100935B0090925700E89507B600FCC6
:10E5C000FDCFC114D10461F0F90140935B00B09319
:10E5D0005700E89507B600FCFDCF79018A01A0E05D
:10E5E000C114D10409F0B5CFB0926601A0926501C3
:10E5F00081E180935700E89529C08091F2009091C5
:10E60000F300892B71F48091E8008B7F8093E80000
:10E6100004C08EB3882309F4E9C08091E80082FF2A
:10E62000F8CF6091F10080916501909166013FD42F
:10E6300080916501909166010196909366018093A7
:10E6400065010150104001151105B9F680E179DD31
:10E650008091E8008B7FBEC08091E800877F809327
:10E66000E80004C08EB3882309F4C0C08091E8009C
:10E6700080FFF8CF80910001893091F08A3069F4F1
:10E6800080916F01813049F480916501909166011C
:10E690008093F1009093F1009AC08091760195C02B
:10E6A0006091670170916801209165013091660168
:10E6B0006F5F7F4FEB01C21BD30B615070408091A5
:10E6C0006F01882389F5D695C795C901A091690185
:10E6D000B0E09C01AD0121C08091F2009091F30067
:10E6E000809771F48091E8008E7F8093E80004C0E9
:10E6F0008EB3882309F47AC08091E80080FFF8CFB8
:10E700004BBFF901879196918093F1009093F100AE
:10E7100021972E5F3F4F4F4F5F4F2097E9F6709341
:10E7200066016093650128C0823031F523C0809175
:10E73000F2009091F300809771F48091E8008E7F51
:10E740008093E80004C08EB3882309F44FC0809101
:10E75000E80080FFF8CF0091650110916601C801C3
:10E760009ED38093F1000F5F1F4F109366010093BB
:10E77000650121972097D9F682E08093000127C098
:10E780008091E800877F8093E80080916A01809300
:10E79000F1001092F1001092F1001092F1008091BE
:10E7A00000018093F1001092F10011C08091E80007
:10E7B000877F8093E80010926A0117C08091E8007B
:10E7C000877F8093E800809100018093F100809121
:10E7D000E8008E7F8093E80008C08091E800877F82
:10E7E0008093E80082E080930001EED0DF91CF912A
:10E7F0001F910F91FF90EF90DF90CF90BF90AF905F
:10E800009F908F9008951F9384B7877F84BF88E17E
:10E810000FB6F89480936000109260000FBE80E005
:10E8200090E020E80FB6F894209361008093610097
:10E830000FBE11E015BF82E085BF41D1569A5E98A8
:10E8400010936F0083E0809381005E9A789401C0FA
:10E850001DD3809101018823D9F780916401882319
:10E86000B9F7D1D056985E9810926F00109281003F
:10E8700081E085BF15BEE0916C01F0916D010995B5
:10E88000FA01923049F0933061F09130F9F488E068
:10E8900091E022E130E01EC08AE191E02BE130E01E
:10E8A00019C0882329F485E391E024E030E012C008
:10E8B000813029F488E990EE28E130E00BC0823005
:10E8C00029F489E391E028E230E004C080E090E0A0
:10E8D00020E030E091838083C90108959B01AC0161
:10E8E00007B600FCFDCFF999FECF83E0F901409314
:10E8F0005B0080935700E89507B600FCFDCF81E1EF
:10E9000080935700E89508959B01AC0107B600FC81
:10E91000FDCFF999FECF85E0F90140935B0080932C
:10E920005700E89507B600FCFDCF81E180935700C2
:10E93000E89508950F931F938B019C0107B600FC87
:10E94000FDCFF999FECF81E00A01F80120935B0029
:10E9500080935700E89511241F910F91089521E2AB
:10E96000FC01209357002491822F089529E0FC0197
:10E97000209357002491822F0895E1E0F0E089E090
:10E980008093570084910895982F07B600FCFDCF1F
:10E99000F999FECF909589E0E1E0F0E0092E8093AF
:10E9A0005700E89508958091EB0081608093EB001B
:10E9B0001092ED006093EC004093ED008091EE002A
:10E9C000881F8827881F08958091790188238CF4F7
:10E9D00003C08EB38823B1F08091E80082FFF9CFA5
:10E9E0008091E8008B7F8093E80008958EB38823A0
:10E9F00049F08091E80080FFF9CF8091E8008E7F98
:10EA00008093E800089564D06BD0E0EEF0E0808160
:10EA100081608083A8EDB0E08C918F778C9319BCD6
:10EA2000E7EDF0E080818E7F80838C918F7E8C93E8
:10EA3000109278010895EF92FF920F931F9348D0A0
:10EA40004FD008ED10E0F80180818F7780838081BE
:10EA50008068808380818F7D8083E7EDF0E0808116
:10EA60008068808319BC1EBA1092770180EEE82E70
:10EA7000F12CF70180818B7F8083F8018081816098
:10EA8000808380E060E042E28EDFE1EEF0E08081B2
:10EA90008E7F8083E2EEF0E08081816080838081E0
:10EAA00088608083F70180818E7F8083F801808178
:10EAB000806180831F910F91FF90EF900895E7EDA3
:10EAC000F0E080818160808381E080937801B3CF22
:10EAD000E8EDF0E080818C7F80831092E200089561
:10EAE0001092DA001092E10008951F920F920FB673
:10EAF0000F920BB60F9211242F933F934F935F9376
:10EB00006F937F938F939F93AF93BF93EF93FF93F5
:10EB10008091DA0080FF1BC08091D80080FF17C071
:10EB20008091DA008E7F8093DA008091D90080FF97
:10EB30000BC084E189BD86E189BD09B400FEFDCF2B
:10EB400081E08EBBA2D103C019BC1EBA9ED18091B8
:10EB5000E10080FF17C08091E20080FF13C0809128
:10EB6000E2008E7F8093E2008091E20080618093DA
:10EB7000E2008091D80080628093D80019BC85E0C3
:10EB80008EBB83D18091E10084FF2CC08091E20094
:10EB900084FF28C084E189BD86E189BD09B400FEF7
:10EBA000FDCF8091D8008F7D8093D8008091E100C7
:10EBB0008F7E8093E1008091E2008F7E8093E2005F
:10EBC0008091E20081608093E20080917701882348
:10EBD00031F48091E30087FD02C081E001C084E050
:10EBE0008EBB53D18091E10083FF21C08091E20070
:10EBF00083FF1DC08091E100877F8093E10082E068
:10EC00008EBB109277018091E1008E7F8093E100AE
:10EC10008091E2008E7F8093E2008091E20080612B
:10EC20008093E20080E060E042E2BDDE2ED1FF9101
:10EC3000EF91BF91AF919F918F917F916F915F9174
:10EC40004F913F912F910F900BBE0F900FBE0F90E1
:10EC50001F9018959C0140917F01509180014617AB
:10EC6000570718F4F90190E03CC06115710511F0E7
:10EC7000AB01F8CF8091E8008E7F8093E80040E000
:10EC800050E0F0CF8EB38823E9F18530E9F180912F
:10EC9000E80083FF02C081E008958091E80082FDD2
:10ECA0002BC08091E80080FF1CC02091F2003091C1
:10ECB000F30007C081918093F100415050402F5FD5
:10ECC0003F4F4115510519F02032310598F390E07E
:10ECD0002032310509F491E08091E8008E7F809325
:10ECE000E8004115510571F6992361F605C08EB310
:10ECF000882341F0853041F08091E80082FFF7CF12
:10ED000080E0089582E0089583E008950F931F93B3
:10ED1000DF93CF9300D0CDB7DEB7E9E7F1E0809184
:10ED2000F100819381E0E138F807C9F766DB809153
:10ED3000E80083FF95C09091790180917A01863037
:10ED400009F441C0873030F4882359F0853009F048
:10ED500087C016C0883009F456C0893009F080C0D9
:10ED600064C0903819F0923809F07AC08091E800B8
:10ED7000877F8093E8001092F1001092F1004EC05E
:10ED8000992309F06DC010917B011F770FB7F8949C
:10ED90008091E800877F8093E80016DE8091E8008C
:10EDA00080FFFCCF8091E3008078812B8093E3008B
:10EDB00080688093E300112311F482E001C083E0B6
:10EDC0008EBB0FBF4DC09058923008F049C0809163
:10EDD0007B0190917C0160917D01AE014F5F5F4F9F
:10EDE0004FDDBC01009709F43BC08091E800877FAC
:10EDF0008093E80089819A812DDF8091E8008B7FE4
:10EE00008093E8002DC0903859F58091E800877F05
:10EE10008093E800809177018093F1008091E80071
:10EE20008E7F8093E800D0DD1BC09923C9F49091B8
:10EE30007B019230A8F48091E800877F8093E800FE
:10EE400090937701C1DD80917701882331F480911F
:10EE5000E30087FD02C081E001C084E08EBB15D0D5
:10EE60008091E80083FF0AC08091EB00806280936C
:10EE7000EB008091E800877F8093E8000F900F906F
:10EE8000CF91DF911F910F91089508958EB388233C
:10EE900029F08091E80083FF01C038CF0895F999E7
:10EEA000FECF92BD81BDF89A992780B50895262F8F
:10EEB000F999FECF1FBA92BD81BD20BD0FB6F8945F
:0EEEC000FA9AF99A0FBE01960895F894FFCFC2
:10EECE0002011E978220DCFB1201100100000020BF
:10EEDE00EB03FB2F00000102000109021B000101E0
:10EEEE000080320904000000FE0102000921030027
:10EEFE0000000C10010403090428034C00550046C1
:10EF0E000041002000440046005500200042006FE2
:10EF1E00006F0074006C006F006100640065007289
:04EF2E0000000000DF
:10FFA0000C946EF40C9484F40C949AF40C94AFF4C6
:10FFB0000C94B6F40C94BDF40C94C4F40895089514
:06FFC00008950895089564
:10FFE000DFCFE0CFE1CFE2CFE3CFE4CFE5CFE6CF85
:08FFF000E6CFE6CFE6CFE6CF35
:08FFF80000E00100B1DFFBDCB9
:040000031000E00009
:00000001FF
